:1000000002EF00F00F0E946E8C6A1F0E956E0F0EAD
:10001000896A926E936A300E8B6E8C8E000000009F
:100020008C9EEBEC00F0EBEC00F08C8E00000000FE
:100030008C9EDAEC00F0DAEC00F08C8E0000000010
:100040008C9EDAEC00F0DAEC00F0200E8B6E8C8ED9
:10005000000000008C9EDAEC00F0DAEC00F0280ED4
:100060000D6E11EC01F0DAEC00F0DAEC00F0080EA5
:100070000D6E11EC01F0DAEC00F0DAEC00F00C0E91
:100080000D6E11EC01F0DAEC00F0DAEC00F0060E87
:100090000D6E11EC01F0DAEC00F0DAEC00F0010E7C
:1000A0000D6E11EC01F0EBEC00F0EBEC00F0030E48
:1000B0000E6E5DEC01F0DAEC00F0480E0E6E36ECE0
:1000C00001F0DAEC00F0650E0E6E36EC01F0DAECC1
:1000D00000F06C0E0E6E36EC01F0DAEC00F06C0EF7
:1000E0000E6E36EC01F0DAEC00F06F0E0E6E36ECB0
:1000F00001F0DAEC00F0200E0E6E36EC01F0DAECD6
:1001000000F04D0E0E6E36EC01F0DAEC00F0430E0E
:100110000E6E36EC01F0DAEC00F0490E0E6E36ECA5
:1001200001F0DAEC00F0500E0E6E36EC01F0DAEC75
:1001300000F0210E0E6E36EC01F0DAEC00F0530EFA
:100140000E6E5DEC01F0DAEC00F03C0E0E6E36EC5B
:1001500001F0DAEC00F03C0E0E6E36EC01F0DAEC59
:1001600000F0630E0E6E5DEC01F0DAEC00F03C0E78
:100170000E6E36EC01F0DAEC00F03C0E0E6E36EC52
:1001800001F0DAEC00F0220E0C6EFEEC00F00C2E0A
:10019000FCD7800E8A6E8A46180E0D6E11EC01F0A7
:1001A0000F0E80140C6E0C2AFEEC00F00C060C6690
:1001B000FBD7F1D7D8CF81F0E8CF80F0E0CF82F045
:1001C000AC0E096E093EFED782C0E0FF80C0E8FF9A
:1001D00081C0D8FF1200D8CF84F0E8CF83F0E0CF01
:1001E00085F0250E0A6EDAEC00F00A2EFCD785C0E9
:1001F000E0FF83C0E8FF84C0D8FF1200D8CF87F0AB
:10020000E8CF86F0E0CF88F0240E0B6EEBEC00F028
:100210000B2EFCD788C0E0FF86C0E8FF87C0D8FF60
:100220001200D8CF8AF0E8CF89F0E0CF8BF00DC074
:100230008BFF8C8E0000000000008C9E8B3A00002B
:1002400000000000000000000000000000000000AE
:10025000000000008C8E0000000000008C9E8BC00F
:10026000E0FF89C0E8FF8AC0D8FF1200D8CF8AF02B
:10027000E8CF89F0E0CF8BF00EC08BFF8C8C8C8E9A
:100280000000000000008C9E8B3A0000000000007F
:10029000000000000000000000000000000000005E
:1002A0008C8E0000000000008C9E8C9C8BC0E0FFB8
:1002B00089C0E8FF8AC0D8FF1200D8CF8AF0E8CF03
:1002C00089F0E0CF8BF0800E0E120EC08BFF8C8E6B
:1002D0000000000000008C9E8B3A0000000000002F
:1002E000000000000000000000000000000000000E
:1002F0008C8E0000000000008C9E8BC0E0FF89C047
:10030000E8FF8AC0D8FF1200FFFFFFFFFFFFFFFFDB
